:020000040000FA
:020000000728CF
:04000A00003400348A
:02000E000730B9
:100010009F008316D73081008B0180308600FF302F
:10002000850083128601142805181428851A3328A0
:10003000051A42285E20363086005E202830860071
:100040005E203A3086005E20113086005E20393016
:1000500086005E20243086005E20353086005E20DB
:1000600052308600142885184428512036308600E6
:1000700051203A30860051203930860051207530A9
:1000800086001428851835285120753086005120A7
:100090003930860051203A308600512036308600B3
:1000A0001428193005197D3085190A30A1008930CE
:1000B000A000A00B5928A10B572808007D30A100F3
:1000C0008930A000A00B6228A10B60280A30A20092
:0600D000A20B68280800E5
:02400E00413F30
:00000001FF
